:100000000C94B3020C94F7020C94F7020C94F702D0
:100010000C94F7020C94F7020C94F7020C94F7027C
:100020000C94F7020C94F7020C94B00D0C94820E11
:100030000C94E01B0C94F7020C94F7020C94F7025A
:100040000C94F7020C94F7020C94F7020C94F7024C
:100050000C94F7020C94481C0C94F7020C94F702D1
:100060000C94F7020C94F7020C94F7020C94F7022C
:100070000C94F7020C94F7020C94F7020C94F7021C
:100080000C94F7020C94F7020C94F7020C94F7020C
:100090000C94F7020C94F7020C94F7020C94F702FC
:1000A0000C94F7020C94F7020C94F702EF0E110F68
:1000B000FF0F110FFF0F560F790FFF0FCE0FE10F3C
:1000C000B012B012DF12DF12151335136614661466
:1000D00040136614F013F01357146614661460147A
:1000E000FD13FD13FD13FD13FD13FD13FD13FD1390
:1000F000FD13FD13FD13FD13FD13FD13FD13FD1380
:100100000F141C1423142A143414750A01E2012C50
:10011000022C02E274FA011602160104020401091B
:1001200002090104020401150215010C020C012848
:10013000022800750A01E2012C022C02E274FA0185
:10014000170217010802080115021501100210011B
:100150000C020C0111021101040204010F020F0133
:1001600028022800750A01E2012C022C02E274FA2E
:100170000105020501050205010802080107020741
:10018000010C020C011702170128022800750A0150
:10019000E30116021602E301E3012B022B02E30145
:1001A000E30115021502E300750A01E301160216C8
:1001B00002E301E3012B022B02E3000000F0A12E79
:1001C000004C002A00E100E00000001E00140004C2
:1001D000001D00E200E2001F001A0016001B00E3F1
:1001E000002A00200008000700060050002C002113
:1001F000001500090019004F004B00220017000AEB
:1002000000050000003500015401520000E3000029
:10021000003400015401520000E3000000290023D3
:10022000001C000B00110000002A00240018000D23
:1002300000100052004E0025000C000E0036005148
:10024000002800260012000F0037002F002B002787
:10025000001300334238713000E0002D00310034CB
:1002600078E5002C00000001000100010001000100
:100270000000003A002F0036020100010001003B9F
:1002800000300037020100010001003C002F02266F
:10029000020100010001003D0030022702010001BF
:1002A0000001003E00340234002E00000001000175
:1002B0000001000000010000000100010001000039
:1002C000000100000001003F0038002D0033020053
:1002D0000001004000240021001E00270001004111
:1002E00000250022001F00370001004200260023E5
:1002F00000200050000100430025022E022E004F76
:10030000000100440045000100010001000000015F
:10031000000100010001000100000069000100016E
:10032000000100010001006A000100043001000129
:1003300000010001004B004E00010001000100011E
:100340000001300100010001004A000100033001FA
:100350000002300000010001000100000001000067
:100360000001001408010000000100000001001A53
:100370000830082F082C0200000100350A520C50EA
:10038000002C00A9004D00350852005100AC00AA15
:100390000019080100510C4F00AB00A8000608012D
:1003A0000001000100010001001B08A5000100AED2
:1003B0000001000100000016034500720067006F95
:1003C0000044006F007800200045005A000000162D
:1003D000034500720067006F0044006F0078002042
:1003E0000045005A0000000403090409026D0004DE
:1003F0000100A0FA09040000010301010009211114
:10040000010001223F000705810308000A090401D9
:10041000000103010200092111010001224D000722
:1004200005820308000A0904020001030000000914
:1004300021110100012236000705830308000A0983
:100440000403000103000000092111010001223909
:1004500000070584031000011201100100000008CC
:10046000EDFE071301000102000105010906A101CB
:10047000050719E029E71500250195087501810296
:100480000508190129059505750191029501750366
:100490009101050719002977150025019578750147
:1004A0008102C005010980A101850216010026B75D
:1004B000001A01002AB700751095018100C0050CD3
:1004C0000901A1018503160100269C021A01002AD8
:1004D0009C02751095018100C005010902A1010966
:1004E00001A10005091901290515002501950575CA
:1004F000018102950175038101050109300931155A
:1005000081257F95027508810609381581257F951B
:100510000175088106050C0A38021581257F9501B1
:1005200075088106C0C005010906A101050719E08B
:1005300029E71500250195087501810295017508C7
:10054000810105081901290595057501910295019B
:10055000750391010507190029FF150025FF950670
:1005600075088100C00011241FBECFEFDAE0DEBFA6
:10057000CDBF04B603FE24C08091F9019091FA0129
:10058000A091FB01B091FC018730904BA740B04B8C
:10059000B9F41092F9011092FA011092FB01109235
:1005A000FC0114BE84B7877F84BF88E10FB6F8943E
:1005B00080936000109260000FBEE0E0FFE30995B9
:1005C00011E0A0E0B1E0E0E2F8E402C005900D9295
:1005D000A433B107D9F711E0A4E3B1E001C01D9243
:1005E000A93FB107E1F70E94F60A0C940E240C947F
:1005F0000000FC016230B9F028F4662341F061305C
:1006000061F023C06330A9F06430C9F01EC082815C
:100610008823D9F088EA91E0089582818823A9F09F
:100620008DE891E008958281882379F084E691E055
:1006300008958281882349F083E391E008958281BF
:10064000882319F08AE091E0089580E090E0089511
:1006500008956091BD017091BE018091BF0190919C
:10066000C0010E94511B56985E9825982D98269897
:100670002E9827982F98813019F0823021F0089514
:10068000259A2D9A0895269A2E9A08950C94290356
:1006900056985E9825982D9826982E9827982F98EA
:1006A0008FEF90E0909389008093880090938B0067
:1006B00080938A0090938D0080938C00259A2D9AC8
:1006C0002FEF80E792E0215080409040E1F700C09A
:1006D0000000269A2E9A2FEF80E792E0215080406A
:1006E0009040E1F700C00000279A2F9A2FEF80E793
:1006F00092E0215080409040E1F700C00000259832
:100700002D982FEF80E792E0215080409040E1F754
:1007100000C0000026982E982FEF80E792E021502D
:1007200080409040E1F700C0000027982F9856982D
:100730005E9825982D9826982E9827982F9808959A
:1007400089EA8093800089E08093810024982C9826
:100750003F988AB18F748AB96E98479A8BB1806B33
:100760008BB9769A0E9448030C94280380E2809308
:1007700000018091340181110EC00E94050481E0C6
:10078000809334012FEF83ED90E32150804090401F
:10079000E1F700C0000080E40E940B048093000198
:1007A00081112EC00E94350480930001811128C060
:1007B0000E94350480930001811122C08FE30E94C2
:1007C00035048093000181111BC00E942D0480E438
:1007D0000E940B0480930001811112C08CE00E94E2
:1007E00035048093000181110BC00E943504809371
:1007F0000001811105C08FE30E9435048093000140
:100800000E942D048091000108951092B9008AE0A1
:100810008093B800089594EA9093BC009091BC0036
:1008200097FFFCCF9091B900987F983021F09031DC
:1008300011F081E008958093BB0084E88093BC00B0
:100840008091BC0087FFFCCF8091B900887F883100
:1008500011F0803471F780E0089584E98093BC0042
:100860008091BC0084FDFCCF08958093BB0084E898
:100870008093BC008091BC0087FFFCCF9091B900B1
:10088000987F81E0983209F480E0089584E88093AD
:10089000BC008091BC0087FFFCCF8091BB00089515
:1008A00080910001811115C080E40E940B048093A7
:1008B000000181110CC082E10E9435048093000187
:1008C000811105C08FEF0E943504809300010E94C2
:1008D0002D0484B1807F84B985B1807F85B98AB1C8
:1008E000837F8AB98BB1837F8BB93E9846980895F0
:1008F0000E94B603809300010E94500480B38C7064
:1009000080BB81B3836F81BBA6E3B1E0E4E4F1E097
:100910008EE08E0F11921D928E13FCCF0C94A003CB
:10092000BF92CF92DF92EF92FF920F931F93CF93DC
:10093000DF9380910001882379F0809135018F5FEA
:1009400080933501811108C00E94B6038093000195
:10095000811102C00E94480306E311E0C0E0D0E02C
:10096000DD24D39482E0C82EEE24E394F12CC7302A
:10097000D10500F580910001811164C080E40E94DE
:100980000B0480930001811112C082E10E943504A2
:100990008093000181110BC0C7010C2E01C0880F8C
:1009A0000A94EAF780950E943504809300010E9422
:1009B0002D0448C0CA30A1F028F4C83059F0C9301D
:1009C00061F005C0CC3089F070F0CD3089F0209A0C
:1009D000289810C0219A29980DC0229A2A980AC0F6
:1009E000239A2B9807C0529A01C0539A5B9802C071
:1009F0003E9A469890EA9A95F1F79FB1799902C08C
:100A000082E001C080E091709D25982B7C9902C006
:100A100084E001C080E0892B7D9902C038E001C0EC
:100A200030E0832B7E9902C020E101C020E0822BC0
:100A30009FB19095991F9927991F9295990F907E34
:100A4000892B0FC080910001811149C080E40E9470
:100A50000B0480930001882379F1B12C0E942D04AE
:100A60008B2DF8019081981719F08083C0920101B5
:100A70000E94500421960F5F1F4FCE30D10509F020
:100A800076CF80910101882361F18150809301012B
:100A9000882339F08FE99FE00197F1F700C000004B
:100AA00020C0A4E4B1E0E6E3F1E0CF01825F9191E0
:100AB0009D938E13FCCF15C083E10E943504809373
:100AC00000018111CACF81E40E940B0480930001D0
:100AD0008111C3CF0E944604B82EB094BFCF80E0EE
:100AE000C0CF0E94460381E0DF91CF911F910F910B
:100AF000FF90EF90DF90CF90BF900895E82FF0E047
:100B0000EC5BFE4F8081089508950F931F93CF9360
:100B1000DF93C4E4D1E010E00C2F025F899190E0F4
:100B20000E94451B180F0C13F9CF812FDF91CF9135
:100B30001F910F91089581E0089581E008950C942C
:100B40009D0508950F931F93CF93DF938C01FC01B4
:100B5000C081D181CE010E94CA19BE010E944B06FC
:100B6000EC01B8010E949F05882309F48DC0F801AB
:100B70008281882309F44AC080915D0181111FC0E0
:100B8000C431F0E5DF0709F051C00E94A10581E002
:100B900080935D010E94121C90935C0180935B0125
:100BA0001092540110925601109255011092580162
:100BB0001092570110925A011092590165C080910C
:100BC0005B0190915C010E941E1C883C910570F4B1
:100BD00080915401E82FF0E0EE0FFF1FEB5AFE4F1B
:100BE000D183C0838F5F809354014EC0C43880E5A9
:100BF000D80721F0C538D04501F13AC0F80182810B
:100C0000882341F01092520182E01EC0C438E0E512
:100C1000DE0759F580915201811106C086E20E94DB
:100C2000541186E20E941C1282E01CC0C438F0E518
:100C3000DF0741F3C538D045D9F4F8018281882314
:100C400031F01092530180E20E946B121DC080911E
:100C50005301811106C087E20E94541187E20E946D
:100C60001C1280E20E9472120FC0C538D04529F3D1
:100C700081E08093520180935301C801DF91CF91AD
:100C80001F910F910C949B0580E0DF91CF911F91F4
:100C90000F910895089596E0799FF001112494E54D
:100CA000899FE00DF11D1124E60FF11DEE0FFF1FCE
:100CB000E154FE4F859194910895880F991FFC018E
:100CC000E55CFF4F859194910895880F991FFC0171
:100CD000E554FE4F8591949108950F931F93CF9300
:100CE000DF93EC018115904350F5C11580E2D807E0
:100CF00008F0C3C0CB3BD10590F4C83AD10508F049
:100D00006AC0C53AD10508F05BC0C430D10508F00F
:100D1000D0C1219709F0CAC101E010E00AC2CF3F5B
:100D2000D10511F008F0C5C1C03FD10508F0A2C03F
:100D3000CE01805E9109089708F4BBC1B7C1C130EC
:100D400090E5D90709F4A2C020F5C0318FE4D80797
:100D500070F4C11590E4D90708F094C0C11521E3DF
:100D6000D20708F0A3C1DD278E01106CE2C1C115C6
:100D7000D04509F09BC10E94D1148FEF94E32CE081
:100D8000815090402040E1F700C000000E946D1C9F
:100D9000D0C1C11597E5D90758F4C03121E5D20774
:100DA00008F01CC1C43180E5D80708F475C07EC1C5
:100DB000CE0190578115904108F078C1DF7073C162
:100DC000C53AD10509F477C1C63AD10509F076C113
:100DD00002E810E4AEC1C83AD10509F472C1C93ABB
:100DE000D10509F471C1CA3AD10509F470C1CB3AF1
:100DF000D10509F46FC1CC3AD10509F46EC1CD3AE1
:100E0000D10509F46DC1C03BD10509F46CC1CE3ADE
:100E1000D10509F46BC1CF3AD10509F46AC1C13BD0
:100E2000D10509F469C1C23BD10509F468C1C33BCE
:100E3000D10509F467C1C43BD10509F466C1C53BBE
:100E4000D10509F465C1C63BD10509F464C1C73BAE
:100E5000D10509F463C1C83BD10509F462C1C93B9E
:100E6000D10509F461C1CA3BD10509F460C100E0B4
:100E700014E45FC18E0110655CC1CE019F700E94B9
:100E8000650658C1DF708E01106A53C18091DA0186
:100E900081608093DA014DC10E94121E811102C04F
:100EA0000E94F81D0E942F1E90E09093F9018093FC
:100EB000F801C23080E5D80721F48091F801816003
:100EC00086C0C43090E5D90721F48091F801826092
:100ED0007EC0C63020E5D20721F48091F8018460FD
:100EE00076C0C83080E5D80719F48091F80127C092
:100EF000CA3090E5D90721F48091F801806167C07C
:100F0000CC3020E5D20721F48091F80180625FC0E7
:100F1000CE3080E5D80721F48091F801806457C075
:100F2000C03190E5D90721F48091F80180684FC065
:100F3000C23120E5D20729F48091F80184608860ED
:100F400046C0C33080E5D80721F48091F8018E7F38
:100F50003EC0C53090E5D90721F48091F8018D7F1E
:100F600036C0C73020E5D20721F48091F8018B7F8D
:100F70002EC0C93080E5D80719F48091F80126C049
:100F8000CB3090E5D90721F48091F8018F7E1FC006
:100F9000CD3020E5D20721F48091F8018F7D17C074
:100FA000CF3080E5D80721F48091F8018F7B0FC006
:100FB000C13190E5D90721F48091F8018F7707C0FE
:100FC000C331D04531F48091F8018B7F877F8093C6
:100FD000F8018091F8010E94331EABC08D2F992734
:100FE0008F70992781309105D9F49E0123703327A2
:100FF00002C0880F991F2A95E2F79C688E0144E091
:10100000000F111F4A95E1F700271370802B912BD9
:1010100053E0CC0FDD1F5A95E1F7C076DD272FC0D6
:101020008230910531F4DC2FCC278E01016F106ADC
:1010300080C08330910569F4CE018370992701E067
:1010400010E002C0000F111F8A95E2F7C8019C68EA
:101050000FC084309105B9F4CE018370992701E067
:1010600010E002C0000F111F8A95E2F7C8019A68CC
:1010700023E0CC0FDD1F2A95E1F7C07ED7708C01ED
:101080000C2B1D2B56C08530910531F4DC2FCC275D
:101090008E01046F106A4DC0069709F04AC0CF71E7
:1010A000DD27DC2FCC278E01106243C000E010E06A
:1010B00040C08E013EC001E810E43BC003E810E4EC
:1010C00038C002EE14E435C009EE14E432C00AEE72
:1010D00014E42FC005EB14E42CC006EB14E429C083
:1010E00007EB14E426C00CEC14E423C00DEC14E46C
:1010F00020C003E815E41DC00AE815E41AC002E99F
:1011000015E417C004E915E414C001E216E411C0A7
:1011100003E216E40EC004E216E40BC005E216E496
:1011200008C006E216E405C007E216E402C00AE2BF
:1011300016E4C801DF91CF911F910F91089596E0B9
:10114000799FF001112494E5899FE00DF11D112490
:10115000E60FF11DEE0FFF1FE154FE4F85919491B4
:10116000803E9105E0F4803C910558F5813391056E
:1011700009F46FC048F48932910509F463C08A32DA
:10118000910509F46DC072C089339105E9F0823888
:101190009105D1F08533910509F44DC067C0833EB8
:1011A000910581F138F4803E9105B9F0823E9105B8
:1011B000D9F05CC0863E910561F1873E9105A1F1B1
:1011C00055C00E945D0608952091F80120FD02C0DF
:1011D00021FF4CC080EE90E049C08091F80180FF73
:1011E000F9CF89E390E042C08091F80182FF0EC000
:1011F0008091F80184FF03C080E090E037C083EE67
:1012000090E034C08091F80182FFF2CF82EE90E04E
:101210002DC08091F80183FF0BC08091F80184FDFF
:10122000EBCF87EE90E022C08091F80183FFF5CFED
:1012300086EE90E01BC08091F80185FF07C089E22F
:1012400090E014C08091F80185FFF9CF85E390E02C
:101250000DC08091F80186FF07C08AE290E006C0C9
:101260008091F80186FFF9CF81E390E00E946D063E
:10127000089508950C94390980916E010895CF93D3
:10128000DF9300D01F92CDB7DEB79C018091EF01B4
:10129000843019F593E099833B832A839093E90086
:1012A0008FEF9091E800815095FD06C095ED9A95DD
:1012B000F1F700008111F5CF8091E80085FF0DC0A6
:1012C00040E050E063E070E0CE0101960E94A00B88
:1012D0008091E8008E778093E8000F900F900F9038
:1012E000DF91CF910895CF93DF9300D01F92CDB7B8
:1012F000DEB72091EF01243021F522E029839B8382
:101300008A8383E08093E9008FEF9091E800815019
:1013100095FD06C095ED9A95F1F700008111F5CF86
:101320008091E80085FF0DC040E050E063E070E090
:10133000CE0101960E94A00B8091E8008E778093E9
:10134000E8000F900F900F90DF91CF9108952091BA
:10135000EF012430F1F422E02093E9002FEF3091E7
:10136000E800215035FD06C035ED3A95F1F7000053
:101370002111F5CF2091E80025FF0BC040E050E09F
:1013800065E070E00E94A00B8091E8008E7780936A
:10139000E8000895CF93DF93EC019091EF01943032
:1013A00009F046C080910C018823D9F080910D018D
:1013B0008823B9F09093E9008FEF9091E800815075
:1013C00095FD06C095E19A95F1F700008111F5CFE2
:1013D0008091E80085FF2CC040E050E060E170E0C3
:1013E00017C081E08093E9008FEF9091E800815071
:1013F00095FD06C095ED9A95F1F700008111F5CFA6
:101400008091E80085FF14C040E050E068E070E0A3
:10141000CE010E94A00B8091E8008E778093E800B7
:1014200080E1FE01AEE5B1E001900D928A95E1F711
:10143000DF91CF9108958091EE01811109C00E9442
:10144000350D0E94920D8091E20084608093E2004D
:1014500008951092EE010895089508950C94DA1BF2
:1014600042E061EC81E00E94AF0C42E061EC82E07E
:101470000E94AF0C42E061EC83E00E94AF0C42E1BD
:1014800061EC84E00C94AF0C8091F101833009F49D
:1014900055C030F4813071F0823009F48EC0089567
:1014A0008A3009F47AC08B3009F460C0893009F0C1
:1014B0009CC020C08091F001813A09F096C08091D3
:1014C000E800877F8093E8008091F4019091F50116
:1014D000892B21F460E18EE591E003C060E080E0BB
:1014E00090E070E00E94EB0B8091E8008B77809396
:1014F000E80008958091F001813209F076C0809172
:10150000F4019091F501009719F0039709F06DC06F
:101510008091E800877F8093E8008091E80082FD59
:1015200005C08091EF018111F8CF5FC08091F1007B
:1015300080936E018091E8008B7753C08091F00119
:10154000813A09F052C08091F4019091F501892B04
:1015500009F04BC08091E800877F8093E80080917C
:10156000E80080FFFCCF80910C0136C08091F00133
:101570008132D9F58091F4019091F501892BA9F57B
:101580008091E800877F8093E8000E94E40C8091BE
:10159000F20180930C010C94D1148091F0018132FE
:1015A00021F58091E800877F8093E8000E94E40C99
:1015B0008091F30180936F0108958091F001813A49
:1015C000A1F48091E800877F8093E8008091E80093
:1015D00080FFFCCF80916F018093F1008091E80043
:1015E0008E778093E8000C94E40C089584B7877F8D
:1015F00084BF88E10FB6F894809360001092600079
:101600000FBE90E080E80FB6F8948093610090934D
:1016100061000FBE0E9487100E94350D0E94920D3E
:101620008091E20084608093E20078940E94181018
:101630000E94891082E091E00E9433108091EF01B6
:10164000853069F40E94A11B8091ED018823B1F3DC
:101650000E94CC1B882391F30E948A0BEFCF0E943B
:101660008F10ECCF292F332723303105C9F064F4D4
:101670002130310581F02230310509F043C08DE67B
:1016800090E02BEE33E042C021323105F1F02232FE
:10169000310541F137C082E190E028E534E036C001
:1016A00099278130910541F08230910541F0892BD5
:1016B00049F5E7EEF3E005C0EFECF3E002C0E7EB3D
:1016C000F3E0849190E09F0121C06430D8F4E62FCC
:1016D000F0E0EE0FFF1FEE5DFE4F2081318189E0CB
:1016E00090E014C0643070F470E0FB01EE0FFF1F57
:1016F000E65EFE4F20813181FB01EA5EFE4F808174
:1017000090E004C080E090E020E030E0FA01318316
:101710002083089580E189BD82E189BD09B400FE7E
:10172000FDCF8091D8008F7D8093D8008091E0001C
:1017300082608093E0008091E00081FDFCCF0895FD
:10174000CF92DF92EF92FF920F931F93CF93DF938D
:10175000EC018B016A010E94030D811133C0C11499
:10176000D10439F0F60180819181081B190BC80F53
:10177000D91FE12CF12C0115110519F18091E80018
:1017800085FD16C08091E8008E778093E800C11433
:10179000D10449F0F60180819181E80EF91EF182B1
:1017A000E08285E00FC00E94030D882321F30AC068
:1017B00089918093F10001501109FFEFEF1AFF0AA0
:1017C000DACF80E0DF91CF911F910F91FF90EF90E2
:1017D000DF90CF9008952091F6013091F701261700
:1017E000370748F06115710539F42091E8002E772C
:1017F0002093E80001C0B90140E061157105A9F12D
:101800002091EF01222309F443C0253009F442C09E
:101810002091E80023FD40C02091E80022FD32C065
:101820002091E80020FFE9CF4091F3002091F200E1
:1018300030E0342BFC01CF016115710559F02830DF
:10184000310540F481918093F100615071092F5F5F
:101850003F4FF1CF41E02830310509F040E02091C1
:10186000E8002E772093E800C8CF4111C9CF0AC005
:101870008091EF01882361F0853061F08091E8006C
:1018800083FD0AC08091E80082FFF2CF80E00895D6
:1018900082E0089583E0089581E008952091F601A3
:1018A0003091F7012617370748F06115710539F4B3
:1018B0002091E8002E772093E80001C0B901FC01D7
:1018C00020E06115710591F18091EF01882309F401
:1018D00040C0853009F43FC08091E80083FD3DC0E1
:1018E0008091E80082FD2FC08091E80080FFE9CF61
:1018F0002091F3008091F20090E0922B6115710528
:1019000059F08830910540F424912093F1003196EC
:10191000615071090196F2CF21E0089709F020E0AB
:101920008091E8008E778093E800CBCF2111CCCF57
:101930000AC08091EF01882361F0853061F08091C9
:10194000E80083FD0AC08091E80082FFF2CF80E0CA
:10195000089582E0089583E0089581E00895982F26
:10196000973058F59093E900981739F07091EC0092
:101970002091ED005091F00003C0242F762F50E00D
:1019800021FF19C03091EB003E7F3093EB00309186
:10199000ED003D7F3093ED003091EB0031603093EE
:1019A000EB007093EC002093ED005093F000209139
:1019B000EE0027FF07C09F5FD3CF8F708093E900B1
:1019C00081E0089580E008958091F00187FF11C0C3
:1019D0008091E80082FD05C08091EF018111F8CF70
:1019E00011C08091E8008B770BC08091EF018823B4
:1019F00049F08091E80080FFF8CF8091E8008E7771
:101A00008093E80008952091E4003091E50095E688
:101A10004091EC00842F817040FF22C08091E8004B
:101A200080FD1CC08091EF01882391F0853091F0FA
:101A30008091EB0085FD10C04091E4005091E500DD
:101A40004217530729F39A01915011F784E0089542
:101A500082E0089583E0089581E0089580E008958C
:101A60004091E80042FFDECF08950E94A30D0E943E
:101A7000AB0DE0EEF0E0808181608083E8EDF0E086
:101A800080818F77808319BCA7EDB0E08C918E7F29
:101A90008C9380818F7E80831092EE0108950F9346
:101AA0001F93CF93DF930E94A30D0E94AB0DC8ED4F
:101AB000D0E088818F778883888180688883888157
:101AC0008F7D888319BC1092EF011092EB01109268
:101AD000ED011092EC0100EE10E0F80180818B7FA7
:101AE000808388818160888342E060E080E00E949A
:101AF000AF0CE1EEF0E080818E7F8083E2EEF0E0DB
:101B0000808181608083808188608083F80180810A
:101B10008E7F8083888180618883DF91CF911F9140
:101B20000F910895E8EDF0E080818F7E8083E7EDEE
:101B3000F0E080818160808384E082BF81E08093D7
:101B4000EE010C944F0DE8EDF0E080818E7F8083F4
:101B50001092E20008951092DA001092E1000895C8
:101B60001F920F920FB60F9211242F933F934F9312
:101B70005F936F937F938F939F93AF93BF93EF93F5
:101B8000FF938091E10082FF0BC08091E20082FF11
:101B900007C08091E1008B7F8093E1000E941710C5
:101BA0008091DA0080FF1FC08091D80080FF1BC0A9
:101BB0008091DA008E7F8093DA008091D90080FFD7
:101BC0000DC080E189BD82E189BD09B400FEFDCF71
:101BD00081E08093EF010E941B0A05C019BC10929E
:101BE000EF010E94290A8091E10080FF19C08091D5
:101BF000E20080FF15C08091E2008E7F8093E200BA
:101C00008091E20080618093E2008091D800806240
:101C10008093D80019BC85E08093EF010E942D0AC3
:101C20008091E10084FF30C08091E20084FF2CC0ED
:101C300080E189BD82E189BD09B400FEFDCF8091BC
:101C4000D8008F7D8093D8008091E1008F7E8093B3
:101C5000E1008091E2008F7E8093E2008091E200BB
:101C600081608093E2008091EB01882311F084E091
:101C700007C08091E30087FD02C081E001C083E0DE
:101C80008093EF010E942E0A8091E10083FF29C01A
:101C90008091E20083FF25C08091E100877F8093DF
:101CA000E10082E08093EF011092EB018091E1006E
:101CB0008E7F8093E1008091E2008E7F8093E2002E
:101CC0008091E20080618093E20042E060E080E089
:101CD0000E94AF0C8091F00088608093F0000E9419
:101CE0002C0AFF91EF91BF91AF919F918F917F91BE
:101CF0006F915F914F913F912F910F900FBE0F9079
:101D00001F9018951F920F920FB60F9211242F93C8
:101D10003F934F935F936F937F938F939F93AF9373
:101D2000BF93CF93DF93EF93FF93C091E900CF7000
:101D30008091EC00D82FD17080FDD0E81092E9009E
:101D40008091F000877F8093F00078940E94C60E07
:101D50001092E9008091F00088608093F000CD2B14
:101D6000CF70C093E900FF91EF91DF91CF91BF91C8
:101D7000AF919F918F917F916F915F914F913F9123
:101D80002F910F900FBE0F901F9018951F93CF9318
:101D9000DF93CDB7DEB7AA970FB6F894DEBF0FBEBC
:101DA000CDBFE0EFF1E088E08E0F9091F1009193CC
:101DB0008E13FBCF0E94440A8091E80083FF1FC16D
:101DC0008091F0019091F101492F50E04A30510586
:101DD00008F015C1FA01EA5AFF4F0C94BE2380386F
:101DE00081F0823809F00BC18091F4018F708093EB
:101DF000E9008091EB0085FB882780F91092E900CB
:101E000006C08091EC019091ED019111826090915A
:101E1000E800977F9093E8008093F1001092F10022
:101E2000C8C0282F2D7F09F0EAC0882319F082301E
:101E300061F0E5C08091F201813009F0E0C093309B
:101E400009F080E08093ED012BC08091F2018111B7
:101E500027C08091F4018F7009F4D1C08093E9000C
:101E60002091EB0020FF1CC0933021F48091EB0007
:101E7000806214C09091EB0090619093EB0021E0A0
:101E800030E0A90102C0440F551F8A95E2F7409344
:101E9000EA001092EA008091EB0088608093EB00EA
:101EA0001092E9008091E800877F86C08111A7C069
:101EB0001091F2011F778091E3008078812B80934D
:101EC000E3008091E800877F8093E8000E94E40CA3
:101ED0008091E80080FFFCCF8091E30080688093D0
:101EE000E300111102C082E001C083E08093EF01A2
:101EF00086C08058823008F082C08091F2019091B3
:101F0000F3018C3D53E0950779F583E08A838AE2FB
:101F100089834FB7F894DE01139620E03EE051E24A
:101F2000E32FF0E050935700E49120FF03C0E295C7
:101F3000EF703F5FEF708E2F90E0EA3010F0C796A1
:101F400001C0C0968D939D932F5F243149F74FBFF9
:101F50008091E800877F8093E8006AE270E0CE011C
:101F600001960E94EB0B14C0AE014F5F5F4F609172
:101F7000F4010E94320BBC01892B09F440C09091FE
:101F8000E800977F9093E80089819A810E944E0C27
:101F90008091E8008B778093E80031C0803879F534
:101FA0008091E800877F8093E8008091EB01809327
:101FB000F1008091E8008E778093E8000E94E40CA5
:101FC0001EC081111CC09091F2019230C0F480912A
:101FD000E800877F8093E8009093EB010E94E40C77
:101FE0008091EB01811106C08091E30087FD02C062
:101FF00081E001C084E08093EF010E94300A80916B
:10200000E80083FF0AC08091E800877F8093E800A2
:102010008091EB0080628093EB00AA960FB6F89453
:10202000DEBF0FBECDBFDF91CF911F910895089500
:10203000CF938091EF018823A1F0C091E900CF7088
:102040009091EC00892F817090FD80E8C82B109250
:10205000E9008091E80083FD0E94C60ECF70C09316
:10206000E900CF91089590937501809374010895CC
:10207000E0917401F0917501309721F00190F081A9
:10208000E02D099480E00895E0917401F0917501CC
:10209000309721F00280F381E02D09940895E091BA
:1020A0007401F0917501309721F00480F581E02DE5
:1020B000099408952091720130917301821793075A
:1020C00071F09093730180937201E0917401F0912B
:1020D0007501309721F00680F781E02D099408956D
:1020E00020917001309171018217930771F09093E4
:1020F000710180937001E0917401F0917501309746
:1021000021F00084F185E02D0994089508950C9440
:1021100086100E94091C0E9478040C94CB1C9F928C
:10212000AF92BF92CF92DF92EF92FF920F931F93E5
:10213000CF93DF9300D000D000D0CDB7DEB70E94A0
:1021400090040DE010E0AA24A394B12C902E802FCF
:102150000E947E05980129583E4F6901F901F080DF
:10216000F826A1F40150110988F78FEF89838A833B
:102170001B820E94121C8160782F9D838C83498171
:102180005A816B818D810E9426112FC09091DA01B6
:1021900091FF04C08E830E9484058E8125E030E08B
:1021A000A501022E01C0440F0A94EAF7E42E4F2144
:1021B000C1F029839A828E2191E009F490E09B83FB
:1021C0000E94121C8160782F9D838C8349815A81E3
:1021D0006B818D810E942611F6018081E826E082C4
:1021E00004C021503109E0F6BDCF0E94B21F10910A
:1021F00076010E9438101817B9F00E9438108093A9
:10220000760126960FB6F894DEBF0FBECDBFDF91E4
:10221000CF911F910F91FF90EF90DF90CF90BF90E3
:10222000AF909F900C943A0926960FB6F894DEBFB3
:102230000FBECDBFDF91CF911F910F91FF90EF9017
:10224000DF90CF90BF90AF909F900895CF93DF9392
:10225000CDB7DEB72B970FB6F894DEBF0FBECDBF5C
:102260004F83588769877A878B87DE01119686E0CE
:10227000FD0111928A95E9F785E0FE0137960190FC
:102280000D928A95E1F749815A816B817C818D811C
:102290009E810E946F172B960FB6F894DEBF0FBE7B
:1022A000CDBFDF91CF910895CF93882309F4C2C0A9
:1022B000C82F823859F40E94381081FDBBC089E3D1
:1022C0000E94491A0E94161B89E30CC0833879F4D6
:1022D0000E94381080FDAEC083E50E94491A0E941A
:1022E000161B83E50E948B1ACF910C94161B843821
:1022F00059F40E94381082FD9DC087E40E94491A5B
:102300000E94161B87E4EECF8CEF8C0F813A48F4C5
:102310008C2F0E94ED2181118DC08C2F0E94491AB3
:10232000E3CF80E28C0F883048F4C77081E001C0B1
:10233000880FCA95EAF70E94CF1AD6CF8BE58C0F8B
:10234000833078F4C53A29F0C63A31F083E890E05A
:1023500005C081E890E002C082E890E0CF910C9443
:102360005A1088E58C0F833108F064C0C83A39F1FF
:10237000C93A41F1CA3A49F1CB3A51F1CC3A59F153
:10238000CD3A61F1C03B69F1CE3A71F1CF3A79F1C2
:10239000C13B81F1C23B89F1C33B91F1C43B99F14F
:1023A000C53BA1F1C63BA9F1C73BB1F1C83BB9F1AF
:1023B000C93BC1F1CA3BC9F180E090E038C082EE70
:1023C00090E035C089EE90E032C08AEE90E02FC0F8
:1023D00085EB90E02CC086EB90E029C087EB90E085
:1023E00026C08CEC90E023C08DEC90E020C083E808
:1023F00091E01DC08AE891E01AC082E991E017C01F
:1024000084E991E014C081E292E011C083E292E09D
:102410000EC084E292E00BC085E292E008C086E242
:1024200092E005C087E292E002C08AE292E0CF919A
:102430000C947010CF910895882309F44BC0823812
:1024400059F40E94381081FF45C089E30E94491A5F
:102450000E94161B89E30CC0833871F40E94381067
:1024600080FF38C083E50E94491A0E94161B83E54D
:102470000E948B1A0C94161B843859F40E94381051
:1024800082FF28C087E40E94491A0E94161B87E435
:10249000EFCF9CEF980F913A58F390E2980F983055
:1024A00050F4877091E001C0990F8A95EAF7892F5F
:1024B0000E94D51ADFCF9BE5980F933020F480E07F
:1024C00090E00C945A10885A833120F480E090E018
:1024D0000C9470100895882321F00E94CF1A0C9458
:1024E000161B0895882321F00E94D51A0C94161B00
:1024F00008957F928F929F92AF92BF92CF92DF9278
:10250000EF92FF920F931F93CF93DF931F92CDB75C
:10251000DEB77C01C62E772EFC01058102950F7077
:10252000128111110E94EC1A0E94421A882379F03C
:10253000112369F080E28C0D883048F082E00E941F
:102540002B1A0E94421A91E0D82ED92601C0D12C14
:10255000E72DE295EF70F0E0E05AFF4F0C94BE23B8
:10256000872D807F072D0F70882311F00295007F43
:10257000112389F0002309F490C180E28C0D88308A
:1025800020F4802F0E94CF1A03C0802F0E94DF1AF0
:102590000E94161B82C18C2D0E941C12002309F47C
:1025A00095C180E28C0D883020F4802F0E94D51ACE
:1025B00003C0802F0E94E51A0E94161B87C1972D29
:1025C000907F872D8F70903211F08295807FCC2084
:1025D00021F0F1E0CF16B1F01EC0112349F0002325
:1025E00009F414C1013009F011C10E94FF1A6EC133
:1025F000002319F0013009F469C189830E94021B8C
:1026000089810AC1112321F0023008F05FC1FEC0A8
:1026100001115CC101C1112321F0002309F4F6C0AE
:102620003CC1002309F4F8C03EC1872D86958695EC
:10263000837090E0009719F0019761F047C1112372
:1026400021F08C2D972D937002C080E090E00E94C5
:102650005A103CC1112321F08C2D972D937002C08C
:1026600080E090E00E94701031C18C2D112319F090
:102670000E94BA1E02C00E94221F0E94A71F26C1EC
:10268000872D837009F052C0111120C18C2D8295C5
:1026900086958770880F880F9C2D9F70892E912CAE
:1026A000A12CB12C082E04C0880C991CAA1CBB1CA0
:1026B0000A94D2F7C4FE14C00FE010E020E030E02E
:1026C000B901A80104C0440F551F661F771F8A95E2
:1026D000D2F7CB01BA01609570958095909503C0B3
:1026E00060E070E0CB01272D26952695237030E021
:1026F0002230310569F02330310589F068297929C4
:102700008A299B292130310571F00E94B718DEC05B
:10271000682979298A299B290E94D318D7C00E9449
:10272000B718C501B4010E949B18D0C0112319F03D
:10273000872D817001C08695882309F4C7C08C2D30
:10274000829586958770880F880F9C2D9F70892EA3
:10275000912CA12CB12C082E04C0880C991CAA1C09
:10276000BB1C0A94D2F7C4FE14C00FE010E020E0B6
:1027700030E0B901A80104C0440F551F661F771F40
:102780008A95D2F7CB01BA016095709580959095A6
:1027900003C060E070E0CB01272D269526952370BD
:1027A000422F50E04230510569F04330510589F025
:1027B000682979298A299B294130510571F00E94A5
:1027C000911984C0682979298A299B290E94AD1909
:1027D0007DC00E949119C501B4010E94751976C08F
:1027E0008C2D90E0FC01E05EF109E531F10508F087
:1027F00050C0E059FF4F0C94BE230C2D0F70872D55
:102800008F71112331F00E940E19802F0E946B12DC
:102810005DC00E942F19802F0E94721257C0112391
:1028200039F0011153C0872D8F710E9454194EC089
:10283000023008F04BC0F7CF112339F0872D8F718C
:102840000E940E1943C01123C9F3872D8F710E9476
:102850002F193CC0112329F0872D8F710E94F91880
:1028600035C00E94EF1832C0112351F0172D1F718F
:10287000812F0E940E1963E0812F0E94221A26C028
:1028800081E00E942B1A023008F182E00E942B1A8C
:102890001DC0112331F0002389F28C2D0E945411A8
:1028A00015C0002391F28C2D0E941C120FC0472DE1
:1028B0004F706C2DC7010E94F9020E94131806C0C8
:1028C000472D4F706C2DC7010E944A06DD20F9F09C
:1028D0000E941E1A80FD1BC0F70112820E94181A66
:1028E0000E940E19C7010E9496140E94181A0F9098
:1028F000DF91CF911F910F91FF90EF90DF90CF90DC
:10290000BF90AF909F908F907F900C942F190F9055
:10291000DF91CF911F910F91FF90EF90DF90CF90BB
:10292000BF90AF909F908F907F9008950F931F93CB
:10293000CF93DF93EC01888199812B813C81232BFC
:10294000B9F09F3F11F48F3F99F0CE010E94A2058C
:10295000882371F0688179818A810E94141A8C0120
:102960000E94C9190E949018B801CE010E947912E4
:10297000DF91CF911F910F9108950E94EC1A0E9450
:10298000FC1A0E94C11A0E94161B0E9458200E9425
:10299000A71F80E090E00E945A1080E090E00C9425
:1029A00070100E94DC1A0C94BD140E94091A292F81
:1029B00022952F7030E02C3031054CF42A3031054F
:1029C0006CF42250310922303105A8F407C02C30B4
:1029D000310569F02F30310551F00DC0803F69F0AD
:1029E00018F4803E40F409C0843F29F406C093FBEC
:1029F000882780F9089580E0089581E00895CF93B5
:102A0000DF9300D000D01F92CDB7DEB70F900F90AC
:102A10000F900F900F90DF91CF910895CF93DF9398
:102A200000D000D000D0CDB7DEB726960FB6F89410
:102A3000DEBF0FBECDBFDF91CF9108951F93CF931F
:102A4000DF93C091850116E080918601C81799F047
:102A5000D0E01C9FF0011D9FF00D1124E957FE4F9F
:102A60004081518162817381848195810E940E151C
:102A70002196C770E9CFDF91CF911F9108954091C2
:102A8000B7015091B8016091B9017091BA0180917C
:102A9000BB019091BC010C940E158091BC018295F4
:102AA0008F7009F054C08091B901882309F44FC098
:102AB00080918501A09186016091B7017091B80164
:102AC0004091BA015091BB01B6E08A1709F43FC0AA
:102AD00090E041155105C1F17F3F11F46F3FA1F125
:102AE000B89FF001B99FF00D1124E957FE4F2181E5
:102AF00072132AC02081621327C02281211124C0B1
:102B0000238134812417350710F421503109241B07
:102B1000350B283C3105C0F42091BC012F70206199
:102B20002093BC0126E0289FF001299FF00D11247D
:102B3000E457FE4F80818F708061808387EB91E046
:102B40000E9496140C941E1501968770BECF0895AE
:102B5000CF92DF92EF92FF920F931F93CF93DF9369
:102B6000CDB7DEB762970FB6F894DEBF0FBECDBF0C
:102B70008C0185E0F801DE011D9601900D928A9589
:102B8000E1F7D8014C9111965C91119712966C91D6
:102B900012971396CD90DC9014973091B7017091F5
:102BA000B8018091BA019091BB01009709F46BC103
:102BB0007F3F19F43F3F09F466C1E090B901EE2070
:102BC00009F4C0C02091BC01C816D90628F0F6014E
:102BD000E81BF90BCF0104C0809590958C0D9D1DCD
:102BE000FF24F394883C910578F0F12C207F09F0C4
:102BF000C6C07C2DD98AC88A89890E94FF1487EBB8
:102C000091E00E949614B1C0822F807F09F046C0E7
:102C1000751314C0341312C0611110C02F702061DD
:102C20002093BC010E943F1587EB91E00E9496140F
:102C30008091BC01D80115968C932EC0CD2819F136
:102C40005F3F11F44F3FF9F0F62E61111CC08091E7
:102C500085012091860136E0821709F45AC090E080
:102C6000389FF001399FF00D1124E957FE4F718113
:102C7000571306C07081471303C07281711103C0DE
:102C800001968770E9CFF62E662309F418C180916A
:102C9000BC0181608093BC01F12C11C1751308C087
:102CA000341306C0611104C08091BC01D801C3C0B7
:102CB0004D875E878D859E856A8B0E94D5146A89B3
:102CC0008823E1F16623D1F12091BC01822F829506
:102CD0008F7090E0029774F08091B7019091B801E5
:102CE00098878F831986DB86CA862C87CE01079644
:102CF0000E94961486E0F801A7EBB1E001900D92D6
:102D00008A95E1F70E944D150E943F15FF24F39428
:102D1000D6C04D875E878D859E850E94091A292F12
:102D200022952F7030E0223031050CF0BCC09F702E
:102D300009F0B6C0805E883008F4C1C0C8010E94A6
:102D40009614E4CFC816D90608F453C0F601E81B60
:102D5000F90BCF01883C910508F450C0F12C7C2D73
:102D6000D98AC88A89890E94FF14E7EBF1E086E0DE
:102D7000DF011D928A95E9F70E943F15A0C07513E7
:102D800014C0341312C0611110C08091BC01F8014D
:102D90008583C8010E94961486E0E7EBF1E0DF012D
:102DA0001D928A95E9F7FE2C8AC04D875E878D8536
:102DB0009E856A8B0E94D5146A89882309F4BECF48
:102DC000662309F4BBCF2091BC01822F82958F70BE
:102DD00090E002970CF48ECF8091B7019091B801EA
:102DE0009A8389831B82DD82CC822E83CE01019659
:102DF0007FCF809590958C0D9D1DACCFF62E6623D0
:102E000009F49CCF75132EC034132CC02091BC0143
:102E100020FD1FC0822F82958F70D9F0D8011596A2
:102E20002C9315978F3049F08F5F982F9295907F54
:102E3000822F8F70892B15968C93C8010E9496144F
:102E400086E0F801A7EBB1E001900D928A95E1F7D9
:102E500093CF86E0F801A7EBB1E001900D928A953F
:102E6000E1F72DC04D875E878D859E850E94D51424
:102E7000811140CF8091BC0181608093BC01C80169
:102E80000E9496141CC0662309F458CF4D875E87B4
:102E90008D859E850E94D514882309F44FCF2ACFB3
:102EA000811148CF0CC0243031050CF047CF9F7002
:102EB00009F440CFF8019581907F09F03BCF8F2D29
:102EC00062960FB6F894DEBF0FBECDBFDF91CF91F3
:102ED0001F910F91FF90EF90DF90CF9008951F9377
:102EE000CF93DF93CDB7DEB72C970FB6F894DEBF44
:102EF0000FBECDBF4F83588769877A878B879C87A2
:102F0000CE0107960E94A815882369F08F819885C5
:102F10002A853B85232BF1F19F3F09F063C08F3F4A
:102F200009F060C037C086E0FE013796DE011196D9
:102F300001900D928A95E1F76F817885EA85FB858E
:102F4000309741F17F3F11F46F3F21F120918601CD
:102F500030E0C9010196877099274091850150E0C2
:102F60008417950709F447C069837A83FD83EC834E
:102F700096E0929FD001939FB00D1124A957BE4FA8
:102F8000FE01319601900D929A95E1F780938601AA
:102F90000E941E1516E08091850190918601891787
:102FA000C1F1189FC001112489579E4F0E94A81596
:102FB000882379F1E09185011E9FF0011124E957E2
:102FC000FE4F4081518162817381848195810E948D
:102FD0000E158091850190E0019687709927809366
:102FE0008501D9CF4F81588569857A858B859C85E8
:102FF0000E940E15CFCF0E94D1141092860110921C
:103000008501E7EBF1E086E0DF011D928A95E9F7A3
:10301000C1CF2C960FB6F894DEBF0FBECDBFDF91A7
:10302000CF911F910895EF92FF920F931F93CF932B
:10303000DF938C01892B09F46CC0F12CEE24E3940E
:10304000E8012196F8018491843740F4843008F037
:1030500051C0813081F0823019F15BC0853709F4AD
:1030600044C0A8F19CE7980F903708F052C08F77C2
:103070000E941C1241C00E5F1F4FFE01C49180E2EE
:103080008C0F883048F4C7708E2D01C0880FCA9508
:10309000EAF70E94EF1A14C08C2F0E9454112DC021
:1030A0000E5F1F4FFE01C49180E28C0F883058F4F0
:1030B000C7708E2D01C0880FCA95EAF70E94F51AD5
:1030C0000E94161B1AC08C2F0E941C1216C00E5F85
:1030D0001F4FFE01C491CC2381F08FE99FE001973F
:1030E000F1F700C00000C150F6CF0E5F1F4FFE0188
:1030F000F49003C00E9454118E018F2D882309F48F
:103100009FCFEFE9FFE03197F1F700C00000815059
:10311000F5CFDF91CF911F910F91FF90EF90089520
:1031200008956093C1017093C2018093C30190938D
:10313000C4010C94BD140F931F930091C101109111
:10314000C2012091C3013091C401DC01CB01802B6D
:10315000912BA22BB32B8093C1019093C201A0931A
:10316000C301B093C4011F910F910C94BD140F9330
:103170001F930091C1011091C2012091C3013091B0
:10318000C401DC01CB0180239123A223B3238093CC
:10319000C1019093C201A093C301B093C4011F91D8
:1031A0000F910C94BD140F931F930091C1011091C6
:1031B000C2012091C3013091C401DC01CB01802701
:1031C0009127A227B3278093C1019093C201A093B6
:1031D000C301B093C4011F910F910C94BD141092C0
:1031E000BD011092BE011092BF011092C0010C945B
:1031F000BD1441E050E060E070E004C0440F551F92
:10320000661F771F8A95D2F74093BD015093BE0188
:103210006093BF017093C0010C94BD1441E050E075
:1032200060E070E004C0440F551F661F771F8A9549
:10323000D2F78091BD019091BE01A091BF01B091E4
:10324000C001482B592B6A2B7B2B4093BD01509317
:10325000BE016093BF017093C0010C94BD1441E0A6
:1032600050E060E070E004C0440F551F661F771FF8
:103270008A95D2F740955095609570958091BD01E3
:103280009091BE01A091BF01B091C0014823592384
:103290006A237B234093BD015093BE016093BF011D
:1032A0007093C0010C94BD1441E050E060E070E008
:1032B00004C0440F551F661F771F8A95D2F780916F
:1032C000BD019091BE01A091BF01B091C0014827FE
:1032D00059276A277B274093BD015093BE01609315
:1032E000BF017093C0010C94BD140F931F93009104
:1032F000BD011091BE012091BF013091C001DC01E0
:10330000CB01802B912BA22BB32B8093BD019093EB
:10331000BE01A093BF01B093C0011F910F910C9407
:10332000BD140F931F930091BD011091BE01209118
:10333000BF013091C001DC01CB0180239123A22386
:10334000B3238093BD019093BE01A093BF01B093BE
:10335000C0011F910F910C94BD140F931F93009106
:10336000BD011091BE012091BF013091C001DC016F
:10337000CB0180279127A227B3278093BD0190938B
:10338000BE01A093BF01B093C0011F910F910C9497
:10339000BD140895CF92DF92EF92FF920F931F9387
:1033A000CF93DF938C01C090C101D090C201E09017
:1033B000C301F090C4018091BD019091BE01A09124
:1033C000BF01B091C001C82AD92AEA2AFB2ACFE15D
:1033D000D0E0D701C6010C2E04C0B695A7959795ED
:1033E00087950A94D2F780FF06C0B8018C2F0E94FF
:1033F0009F08019721F4219760F780E001C08C2F8E
:10340000DF91CF911F910F91FF90EF90DF90CF90C0
:103410000895CF93DF93EC010E94CA19BE010E9468
:103420009F08DF91CF910895CB010E94091A08955A
:103430008091C50185958595859508958091C501F3
:103440008770089598E0899F90011124262B20937E
:10345000C5010C940E192091C5018095822380939B
:10346000C501982F977069F430E0482F552747FD24
:1034700050952417350729F08595859585950C94E9
:103480002F1908959091C501977081E009F480E0AB
:10349000089590910C01992321F090910D019111C3
:1034A00009C020910E0130910F01F90132969FEF72
:1034B00040E01FC0982F9695969596959F3050F5B1
:1034C000E0910E01F0910F01E90FF11D877021E0ED
:1034D00030E0A90102C0440F551F8A95E2F7CA01E6
:1034E0009181892B818308959F3F39F04F5F4E3042
:1034F00041F051915813F8CF0DC05111F7CF942FCF
:10350000F5CF9F3F39F0F901E90FF11D97FDFA95CD
:1035100082830895089590910C01992321F0909150
:103520000D01911109C020910E0130910F01F90197
:103530003296205F3F4F1FC0982F9695969596958F
:103540009F30F0F4E0910E01F0910F01E90FF11DB1
:10355000877021E030E0A90102C0440F551F8A9511
:10356000E2F7CA018095918189238183089531967C
:10357000E217F30729F090819813F9CF1082F7CF63
:10358000089581E090E0E0910E01F0910F01E80FC5
:10359000F91F1082019680319105A9F70895909145
:1035A000D901892B8093D901089580959091D901F3
:1035B00089238093D90108951092D901089590919B
:1035C000D801892B8093D801089580959091D801D6
:1035D00089238093D80108951092D801089590917D
:1035E000D701892B8093D701089580959091D701B9
:1035F00089238093D70108951092D701089580936D
:10360000C60108951092C601089580910E0190910F
:103610000F01FC0131969C01205F3F4F80E09191AA
:1036200091118F5FE217F307D1F70895E0910E0132
:10363000F0910F018091D9018083E0910E01F0910A
:103640000F0190818091D801892B8083E0910E0138
:10365000F0910F0190818091D701892B8083809117
:10366000C601882361F0E0910E01F0910F01908175
:10367000892B80830E94051B81111092C6018091C5
:103680000E0190910F010C94441020E0009739F046
:10369000AC0141505109842395232F5FF7CF822F2E
:1036A0000895CF92DF92EF92FF926C01EE24FF24F7
:1036B000C114D104E104F10421F0C701B60120E1F5
:1036C00001C020E0C72ED82EE92EFF24C114D1045A
:1036D000E104F10419F0285FC701B6016B017C0118
:1036E00054E0F694E794D794C7945A95D1F7C1144F
:1036F000D104E104F10419F02C5FC701B6016B019C
:103700007C0142E0F694E794D794C7944A95D1F7A8
:10371000C114D104E104F10419F02E5FC701B60110
:10372000DC01CB01B695A79597958795892B8A2BB8
:103730008B2B09F02F5F822FFF90EF90DF90CF90BF
:1037400008958091EF01843021F11092DB0120E493
:1037500088E190E00FB6F894A895809360000FBEC2
:103760002093600080E00E943A0983B7817F8460E3
:1037700083BF83B7816083BF7894889583B78E7F3A
:1037800083BF88E10FB6F8948093600010926000C8
:103790000FBE0895089508950E94CA1B0E949004C8
:1037A0000E94CB1B0E94850591E0811101C090E031
:1037B000892F08950E94D1140E9438100C943A0960
:1037C0001F920F920FB60F9211248F939F93AF9376
:1037D000BF938091DB01811113C08091DC01909136
:1037E000DD01A091DE01B091DF014196A11DB11D67
:1037F0008093DC019093DD01A093DE01B093DF01A3
:10380000BF91AF919F918F910F900FBE0F901F901E
:10381000189582E084BD93E095BD9AEF97BD8093A3
:103820006E0008952FB7F8948091DC019091DD012E
:10383000A091DE01B091DF012FBF0895CF92DF92FA
:10384000EF92FF920F931F932FB7F8944091DC01F2
:103850005091DD016091DE017091DF012FBF6A019F
:103860007B01EE24FF248C0120E030E0C016D1065D
:10387000E206F30610F4415051099A01281B390B56
:10388000C9011F910F91FF90EF90DF90CF900895A5
:103890001F920F920FB60F9211248F939F93AF93A5
:1038A000BF938091DC019091DD01A091DE01B09188
:1038B000DF010196A11DB11D8093DC019093DD0114
:1038C000A093DE01B093DF01BF91AF919F918F91E3
:1038D0000F900FBE0F901F9018950E94350DF89411
:1038E0002FEF87EA91E6215080409040E1F700C039
:1038F000000087E090EBDC018093F9019093FA01DE
:10390000A093FB01B093FC019CE088E10FB6F89412
:10391000A895809360000FBE90936000FFCFEF9258
:10392000FF920F931F93CF93DF93D82FCDE08C2F6F
:103930000E947E0505E010E0E82EF12CC701002E64
:1039400002C0959587950A94E2F780FF09C0602F21
:103950007C2F80E00E944B06D81302C081E006C095
:103960000150110958F7C15010F780E0DF91CF9155
:103970001F910F91FF90EF900895CF93C82F8CE285
:103980000E948F1C882321F08C2FCF910C948F1CC8
:1039900080E0CF910895CF930E94121E811102C042
:1039A0000E94F81DC5E6C15049F00E9490048FE3C3
:1039B0009CE90197F1F700C00000F5CF89E20E9471
:1039C000BD1C811113C18AE20E94BD1C81110E949D
:1039D000F81D85E00E94BD1C81110E946D1C0E9493
:1039E0001D1E8093DA0187E00E94BD1C8823A9F187
:1039F0008BE10E94BD1C882351F08091DA0181FB8C
:103A0000222720F991E0922790FB81F90EC08EE0E9
:103A10000E94BD1C882361F08091DA0182FB22277D
:103A200020F991E0922790FB82F98093DA0115C08A
:103A300080E10E94BD1C9091DA01882341F093FB44
:103A4000222720F981E0822780FB93F904C0892F87
:103A5000809580FB90F99093DA018091DA010E94C1
:103A6000211E0E942F1E8093F80180EE0E94BD1C33
:103A7000882341F08091F801982F909590FB80F970
:103A80008093F80189E30E94BD1C882359F080913E
:103A9000F80181FB222720F991E0922790FB81F920
:103AA0008093F80182EE0E94BD1C882359F080911A
:103AB000F80182FB222720F991E0922790FB82F9FE
:103AC0008093F80186EE0E94BD1C882359F08091F6
:103AD000F80183FB222720F991E0922790FB83F9DC
:103AE0008093F80183EE0E94BD1C882359F08091D9
:103AF000F80184FB222720F991E0922790FB84F9BA
:103B00008093F80185E30E94BD1C882359F08091C1
:103B1000F80185FB222720F991E0922790FB85F997
:103B20008093F80181E30E94BD1C882359F08091A5
:103B3000F80186FB222720F991E0922790FB86F975
:103B40008093F80181E10E94BD1C882359F0809187
:103B5000F80187FB222720F991E0922790FB87F953
:103B60008093F8018091F8010E94331E8091F80142
:103B700087FB882780F980930D0187E20E94BD1C96
:103B8000C82F8EE10E94BD1C8111C2608FE10E948E
:103B9000BD1C8111C46080E20E94BD1C8111C860FF
:103BA00081E20E94BD1C8111C06182E20E94BD1CA5
:103BB0008111C06283E20E94BD1C8111C06484E255
:103BC0000E94BD1C882311F0C06802C0CC2329F0DC
:103BD0008C2F0E942A1E6C2F03C00E94261E682F65
:103BE00070E080E090E0CF910C949118CF9108950F
:103BF0006DEE7EEF80E090E00E94F82360E082E0CE
:103C000090E00E94E62360E083E090E00E94E623DB
:103C100060E084E090E00E94E62360E085E090E0D0
:103C20000C94E62380E090E00E94E02321E08D3EAA
:103C30009E4F09F020E0822F089582E090E00C94DE
:103C4000D823682F82E090E00C94E62383E090E094
:103C50000C94D823682F83E090E00C94E62384E052
:103C600090E00C94D823682F84E090E00C94E62335
:103C70008091E20180FF0BC06091130185E0689F95
:103C8000B001112475956795759567952BC081FFD7
:103C900009C06091130185E0689FB00111247595FA
:103CA000679520C082FF07C06091130185E0689F7F
:103CB000B001112417C09091E3019923D1F06091D4
:103CC0001201961788F72091130185E0289F900133
:103CD0001124929FA001939F500D112470E0CA01FE
:103CE0000E94AA236038710540F46115710539F00E
:103CF00002C065E070E0862F08958FE7089581E0A7
:103D000008958091E20180FF08C06091110170E088
:103D1000759567957595679521C081FF06C060917F
:103D2000110170E07595679519C082FF04C060911C
:103D3000110170E010C09091E3019923C1F06091EE
:103D400010019617A0F780911101899FC0011124DD
:103D500070E00E94AA236038710528F4611571058E
:103D600021F0862F08958FE7089581E0089561E09E
:103D700070E0F4CF803F21F40E94381E819504C08A
:103D8000813F29F40E94381E8093E6010895823F06
:103D900021F40E94381E819504C0833F29F40E94BB
:103DA000381E8093E5010895893F19F40E94811E11
:103DB00005C08A3F31F40E94811E81958093E701FE
:103DC00008958B3F21F40E94811E819504C08C3F91
:103DD00029F40E94811E8093E8010895843F21F414
:103DE0008091E401816017C0853F21F48091E40156
:103DF000826011C0863F21F48091E40184600BC091
:103E0000873F21F48091E401886005C0883F31F448
:103E10008091E40180618093E40108958D3F21F455
:103E20008091E20181600BC08E3F21F48091E2011C
:103E3000826005C08F3F29F48091E2018460809305
:103E4000E2010895803F39F48091E60187FF6CC05C
:103E50001092E60169C0813F29F48091E6011816AD
:103E6000BCF362C09091E501823F29F497FF5CC0EA
:103E70001092E50159C0833F19F41916CCF354C0D0
:103E8000893F41F48091E70118160CF04DC0109263
:103E9000E7014AC08A3F29F48091E70187FF44C0C7
:103EA000F6CF8B3F39F48091E80187FF3DC0109237
:103EB000E8013AC08C3F29F48091E8011816BCF360
:103EC00033C0843F21F48091E4018E7F17C0853F89
:103ED00021F48091E4018D7F11C0863F21F480910F
:103EE000E4018B7F0BC0873F21F48091E401877F41
:103EF00005C0883F31F48091E4018F7E8093E40116
:103F000013C08D3F21F48091E2018E7F0BC08E3F64
:103F100021F48091E2018D7F05C08F3F29F48091CB
:103F2000E2018B7F8093E2018091E50181110EC057
:103F30008091E60181110AC08091E701811106C0DC
:103F40008091E801811102C01092E301089584EE8E
:103F500091E00E944F100E94121C9093E101809307
:103F6000E00108951F93CF93DF938091E00190913A
:103F7000E1010E941E1CAC019091E301992321F004
:103F80002091140130E006C0209115018AE0289F9D
:103F9000900111244217530708F486C08091E5016F
:103FA000C091E601D091E7011091E801811107C0AD
:103FB000C11176C0D11174C0111172C075C09F3F7C
:103FC00019F09F5F9093E301181624F40E94381EA5
:103FD0008093E5018091E50187FF05C00E94381EAE
:103FE00081958093E5011C1624F40E94381E80936D
:103FF000E6018091E60187FF05C00E94381E819589
:104000008093E6016091E501662339F1C091E601F4
:10401000CC2319F1772767FD7095872F972F0E9482
:10402000BB2223E333E343E35FE30E941F230E94A9
:1040300088226093E5016C2F772767FD7095872FA5
:10404000972F0E94BB2223E333E343E35FE30E9405
:104050001F230E9488226093E6011D1624F40E940B
:10406000811E8093E7018091E70187FF05C00E94D0
:10407000811E81958093E701111624F40E94811E10
:104080008093E8018091E80187FF05C00E94811EAE
:1040900081958093E801DF91CF911F910C94A71F28
:1040A0009F3F09F08ECF96CFDF91CF911F9108955A
:1040B000E4EEF1E085E0DF011D928A95E9F71092C8
:1040C000E3011092E2010895833081F128F48130F8
:1040D00059F08230D1F00895853009F449C0B8F123
:1040E000863009F456C0089580911501262F30E0DE
:1040F000280F311D2F3F310524F4680F60931501FF
:1041000008958FEF80931501089580911401262F53
:1041100030E0280F311D2F3F310524F4680F6093E4
:10412000140108958FEF8093140108958091130175
:10413000262F30E0280F311D2F3F310524F4680F62
:104140006093130108958FEF809313010895809178
:104150001201262F30E0280F311D2F3F310524F4A6
:10416000680F6093120108958FEF809312010895F4
:1041700080911101262F30E0280F311D2F3F31058E
:1041800024F4680F6093110108958FEF809311015B
:10419000089580911001262F30E0280F311D2F3F08
:1041A000310524F4680F6093100108958FEF809318
:1041B00010010895833011F128F4813049F08230E4
:1041C00091F00895853081F120F18630C1F1089594
:1041D00080911501681720F4861B809315010895BE
:1041E00010921501089580911401681720F4861B20
:1041F0008093140108951092140108958091130181
:10420000681720F4861B8093130108951092130100
:10421000089580911201681720F4861B8093120183
:10422000089510921201089580911101681720F4E9
:10423000861B8093110108951092110108958091B9
:104240001001681720F4861B8093100108951092C6
:10425000100108950F931F938B3109F475C0A0F5D9
:104260008E3009F484C0C0F4873009F45BC068F470
:10427000863009F0AAC08091DA01817F8E7F809319
:10428000DA0181E08093EA01A1C0883009F496C088
:104290008B3009F493C099C0813109F472C068F47D
:1042A000803109F092C08091DA0183FB222720F946
:1042B00091E0922790FB83F950C0863109F47EC0CB
:1042C000893109F47BC081C0853309F479C068F471
:1042D000873209F475C028F48E3108F476C08D5108
:1042E0005AC0893209F46CC070C0833438F48A3300
:1042F00008F050C0883309F461C067C0833409F402
:104300005FC0883409F061C00E94D1140FEF13ED33
:1043100020E3015010402040E1F700C000000E945F
:104320006D1C4CC09091DA01892F8095817080FBC3
:1043300090F929F0966098609093DA0147C0997FD0
:10434000977F9093DA013AC08091DA0181FB2227AE
:1043500020F991E0922790FB81F98093DA0199236B
:1043600069F18091DA0181608093DA0127C0809140
:10437000DA0182FB222720F991E0922790FB82F953
:10438000ECCF0E94D11490910D0181E08927809398
:104390000D0114C0895341E050E060E070E08A01F3
:1043A0009B0104C0000F111F221F331F8A95D2F7F3
:1043B000C901B8010E9491180E94D11481E006C081
:1043C00061E070E080E090E0F5CF80E01F910F9118
:1043D000089580E0089580E00895CF93C82F8091DC
:1043E000EA01813079F018F08230E9F187C0E0917C
:1043F0000E01F0910F018081813169F0823209F064
:104400007FC009C0E0910E01F0910F0180818131E0
:1044100011F0823261F48C2F0E94E921811104C0D5
:104420008C2F0E942A211DC081E090E01AC08C2FA1
:104430000E94EB21811114C0C43179F048F4CB30D3
:1044400079F0C03109F060C082E08093EA0108C0D1
:10445000C93219F0C83321F057C01092EA0154C094
:1044600081E0817053C0C93289F118F5C43171F10E
:10447000A8F4C73009F046C08AE08093150194E1A2
:104480009093140193E0909313018093120188E0BC
:104490008093110188E28093100134C0CE51C63060
:1044A00088F5EC2FF0E0E65DFE4F80818093E90116
:1044B00029C0CE34E9F020F4CB3421F56AE013C0F2
:1044C000C13579F0C235F1F461E00DC08091E901A8
:1044D000882319F01092E90115C081E08093EA0168
:1044E00015C061E006C08091E9010E9464200AC005
:1044F0006AE08091E9010E94DA2004C01092EA018A
:1045000080E004C081E002C080E0ABCFCF9108958D
:1045100004D06894B1118DC0089570D088F09F5771
:1045200090F0B92F9927B751A0F0D1F0660F771FFF
:10453000881F991F1AF0BA95C9F712C0B13081F0DF
:1045400077D0B1E0089574C0672F782F8827B85FBF
:1045500039F0B93FCCF3869577956795B395D9F740
:104560003EF490958095709561957F4F8F4F9F4F4A
:104570000895E89409C097FB3EF490958095709556
:1045800061957F4F8F4F9F4F9923A9F0F92F96E99F
:10459000BB279395F695879577956795B795F11114
:1045A000F8CFFAF4BB0F11F460FF1BC06F5F7F4FB1
:1045B0008F4F9F4F16C0882311F096E911C07723C3
:1045C00021F09EE8872F762F05C0662371F096E8CC
:1045D000862F70E060E02AF09A95660F771F881F9B
:1045E000DAF7880F9695879597F9089557FD9058B3
:1045F000440F551F59F05F3F71F04795880F97FBA7
:10460000991F61F09F3F79F0879508951216130660
:104610001406551FF2CF4695F1DF08C0161617068F
:104620001806991FF1CF86957105610508940895C4
:10463000E894BB2766277727CB0197F908950BD01D
:1046400078C069D028F06ED018F0952309F05AC0D0
:104650005FC01124EECFCADFA0F3959FD1F3950F71
:1046600050E0551F629FF001729FBB27F00DB11DF6
:10467000639FAA27F00DB11DAA1F649F6627B00D86
:10468000A11D661F829F2227B00DA11D621F739F6F
:10469000B00DA11D621F839FA00D611D221F749F7D
:1046A0003327A00D611D231F849F600D211D822FC4
:1046B000762F6A2F11249F5750408AF0E1F088230B
:1046C0004AF0EE0FFF1FBB1F661F771F881F915018
:1046D0005040A9F79E3F510570F014C0AACF5F3F2C
:1046E000ECF3983EDCF3869577956795B795F7954B
:1046F000E7959F5FC1F7FE2B880F911D96958795D3
:1047000097F9089597F99F6780E870E060E0089551
:104710009FEF80EC089500240A94161617061806D9
:104720000906089500240A941216130614060506B5
:104730000895092E0394000C11F4882352F0BB0F46
:1047400040F4BF2B11F460FF04C06F5F7F4F8F4FA9
:104750009F4F089597FB072E16F4009407D077FD1E
:1047600009D00E94C42307FC05D03EF490958195A2
:104770009F4F0895709561957F4F0895EE0FFF1F2D
:104780000590F491E02D0994AA1BBB1B51E107C0D1
:10479000AA1FBB1FA617B70710F0A61BB70B881FD1
:1047A000991F5A95A9F780959095BC01CD01089560
:1047B000F999FECF92BD81BDF89A992780B50895E9
:1047C000A8E1B0E042E050E00C940024262FF999D3
:1047D000FECF92BD81BDF89A019700B4021639F060
:1047E0001FBA20BD0FB6F894FA9AF99A0FBE089531
:1047F0000196272F0E94E7230C94E623DC01CB01CE
:10480000FC01F999FECF06C0F2BDE1BDF89A3196E0
:1048100000B40D9241505040B8F70895F894FFCF7E
:1048200020023C09CA09A70973093F090101C70110
:1048300028080A03140A3F4D36392605D904A30473
:104840006A04FD0316042F0448040102030405064C
:04485000070809004C
:00000001FF
